:100000000AC024C023C022C03DC027C01FC01EC0DC
:100010008BC01CC01BC011271FBFCFE5D0E0DEBFC7
:10002000CDBF20E0A0E4B0E0EAEDF3E402C03191FE
:100030003D93A234B207D9F720E0A2E4B0E001C0BA
:100040001D93A535B207E1F770D0C5C1D9CF00C067
:1000500000C08150910BD8F708951F930F930FB7ED
:100060000F9310E04F9345A14D7F09F4129845A1DD
:100070004150423008F411984F910F910FBF0F91EA
:100080001F9118951F930F930FB70F9310E04F9385
:1000900045A14D7F09F4129A45A14150423008F420
:1000A000119A4F910F910FBF0F911F91189542E038
:1000B0004EBD4BBD48EE53E053BD42BD4AE14DBD80
:1000C00008950898109845B74D7F45BF1BBB80E643
:1000D0009AEEBDDF47E84DBBEE9AEC9BFECF40E1C8
:1000E0004DBBEF9845B7426045BF089A10980895F8
:1000F0009FEF980F8823B9F067E050E0E62FF0E01B
:10010000E65BFF4F4081742F771F7727771F440FDF
:10011000452B40836150572F6F3F81F741A3742BCC
:1001200071AB915048F70895189548ED4CBF16BF34
:100130004FE047BBF894BBDF4BB543604BBD0A9A19
:10014000099A089A789446E040A9BBDFC0A1AC2F79
:10015000B0E0A65BBF4FAF5FBF4FEC91A150B04086
:10016000F0E0F05CE08149B3E40FEC93E37044A16C
:10017000E427E4A94FEF4C0F40A9C113E6CFE330C9
:1001800019F446E142AB02C04EE142AB4AA146A996
:1001900010A94C2F4D3388F066A170E080E490E008
:1001A000E82FF92FE41BF10B862F972F02C09595AE
:1001B0008795EA95E2F784AB02C04AA144AB42A31B
:1001C00050E064A3677002C0559547956A95E2F7C1
:1001D00040FF04C04AA144604AA903C04AA14B7F22
:1001E0004AA944A145A9433009F47DC04AA14695D6
:1001F0004695437009F075C043A14F5F43A952A1D2
:10020000451720F4473008F0C0C078C04513C0C07F
:10021000473010F042E045A941E050E057BD46BDEF
:1002200049E043AB46B557B5440F551F57BD46BDD2
:100230008FEF9FEF0CDF43A35FEF540F53AB4113DE
:10024000F1CF43A152A1541708F0A9C042A9E3A1DC
:10025000E770F0E0E65BFF4F808165E0B0D093ABE4
:100260004EEF50E058A947A961E07FEF42B1462721
:1002700042B943A350E04F5F5F4F542F5295507FD8
:10028000541B550F4FEF450F49A9552329F000C0C6
:1002900000C04150E0F779A947A158A1842F952FBC
:1002A0008150910B98A987A9452B01F780E69AEE1A
:1002B000CEDE43A15FEF540F53A94113C8CF49E0ED
:1002C00043AB46B557B55695479557BD46BD8FEFDD
:1002D0009FEFBDDE43A35FEF540F53AB4113F1CF4C
:1002E0000DC013A90BC04AA142FF03C01298119A76
:1002F00002C0129A119884E89CE1A9DE81E0F8DE40
:1003000040A14F5F40A9403408F444CF53C042B1EC
:10031000462742B925E82A95F1F7000047A158A1E0
:10032000842F952F8150910B98A987A9452B79F798
:100330008FE3DEDE44A1433009F428CFA89559E2CB
:1003400048ED0FB7F894A8954CBF51BF0FBF41B708
:10035000406441BF4AB7417F44604ABF4AB74160E9
:100360004ABF4FB77894889558ED60E00FB7F8947E
:10037000A8955CBF61B7677F61BF0FBF4FBF4AB72A
:100380004E7F4ABF4FE047BB01CF451345CF42CF19
:1003900041E050E057BD46BD49E043AB43CF49E0A3
:1003A00043AB8FCF1298119847ED57E258A947A950
:1003B00061E0ADCF44A1433009F0BACFF3CF991B30
:1003C00079E004C0991F961708F0961B881F7A954C
:0A03D000C9F780950895F894FFCF57
:0203DA0007001A
:00000001FF
